BL51 BANKED LINKER/LOCATER V5.01                                                        11/28/2003  21:21:30  PAGE 1


BL51 BANKED LINKER/LOCATER V5.01, INVOKED BY:
D:\SOFTWARE\EESOFT\KEIL6\C51\BIN\BL51.EXE .\OS_CPU_C.obj, .\OS_CPU_A.obj, .\STARTUP.obj, .\OS_CORE.obj, .\OS_MBOX.obj, .
>> \OS_MEM.obj, .\OS_Q.obj, .\OS_SEM.obj, .\OS_TASK.obj, .\OS_TIME.obj, ex1.obj TO ex1 RAMSIZE (256) XDATA (0X0000-0X7FF
>> F)


MEMORY MODEL: SMALL


INPUT MODULES INCLUDED:
  .\OS_CPU_C.obj (OS_CPU_C)
  .\OS_CPU_A.obj (OS_CPU_A)
  .\STARTUP.obj (?C_STARTUP)
  .\OS_CORE.obj (OS_CORE)
  .\OS_MBOX.obj (OS_MBOX)
  .\OS_MEM.obj (OS_MEM)
  .\OS_Q.obj (OS_Q)
  .\OS_SEM.obj (OS_SEM)
  .\OS_TASK.obj (OS_TASK)
  .\OS_TIME.obj (OS_TIME)
  ex1.obj (EX1)
  D:\SOFTWARE\EESOFT\KEIL6\C51\LIB\C51S.LIB (?C_INIT)
  D:\SOFTWARE\EESOFT\KEIL6\C51\LIB\C51S.LIB (?C?COPY)
  D:\SOFTWARE\EESOFT\KEIL6\C51\LIB\C51S.LIB (?C?IILDX)
  D:\SOFTWARE\EESOFT\KEIL6\C51\LIB\C51S.LIB (?C?LMUL)
  D:\SOFTWARE\EESOFT\KEIL6\C51\LIB\C51S.LIB (?C?ULDIV)
  D:\SOFTWARE\EESOFT\KEIL6\C51\LIB\C51S.LIB (?C?LLDIDATA)
  D:\SOFTWARE\EESOFT\KEIL6\C51\LIB\C51S.LIB (?C?LSTIDATA)
  D:\SOFTWARE\EESOFT\KEIL6\C51\LIB\C51S.LIB (?C?LSTXDATA)
  D:\SOFTWARE\EESOFT\KEIL6\C51\LIB\C51S.LIB (?C?LSTKXDATA)
  D:\SOFTWARE\EESOFT\KEIL6\C51\LIB\C51S.LIB (?C?OFFXADD)
  D:\SOFTWARE\EESOFT\KEIL6\C51\LIB\C51S.LIB (?C_IBP)
  D:\SOFTWARE\EESOFT\KEIL6\C51\LIB\C51S.LIB (PRINTF)
  D:\SOFTWARE\EESOFT\KEIL6\C51\LIB\C51S.LIB (?C?CLDPTR)
  D:\SOFTWARE\EESOFT\KEIL6\C51\LIB\C51S.LIB (?C?CLDOPTR)
  D:\SOFTWARE\EESOFT\KEIL6\C51\LIB\C51S.LIB (?C?CSTPTR)
  D:\SOFTWARE\EESOFT\KEIL6\C51\LIB\C51S.LIB (?C?PLDIIDATA)
  D:\SOFTWARE\EESOFT\KEIL6\C51\LIB\C51S.LIB (?C?CCASE)
  D:\SOFTWARE\EESOFT\KEIL6\C51\LIB\C51S.LIB (PUTCHAR)


LINK MAP OF MODULE:  ex1 (OS_CPU_C)


            TYPE    BASE      LENGTH    RELOCATION   SEGMENT NAME
            -----------------------------------------------------

            * * * * * * *   D A T A   M E M O R Y   * * * * * * *
            REG     0000H     0008H     ABSOLUTE     "REG BANK 0"
            DATA    0008H     0014H     UNIT         _DATA_GROUP_
            DATA    001CH     0001H     UNIT         ?C?LIB_DATA
                    001DH     0003H                  *** GAP ***
            BIT     0020H.0   0001H.1   UNIT         _BIT_GROUP_
                    0021H.1   0000H.7                *** GAP ***
            IDATA   0022H     0001H     UNIT         ?STACK

            * * * * * * *  X D A T A   M E M O R Y  * * * * * * *
            XDATA   0000H     03E8H     UNIT         ?XD?OS_CORE
BL51 BANKED LINKER/LOCATER V5.01                                                      11/28/2003  21:21:30  PAGE 2


            XDATA   03E8H     01F0H     UNIT         ?XD?EX1

            * * * * * * *   C O D E   M E M O R Y   * * * * * * *
            CODE    0000H     0003H     ABSOLUTE     
            CODE    0003H     0005H     UNIT         ?PR?_?OSVERSION?OS_CORE
            CODE    0008H     0001H     UNIT         ?PR?_?OSTASKSWHOOK?OS_CPU_C
            CODE    0009H     0001H     UNIT         ?PR?_?OSTASKSTATHOOK?OS_CPU_C
            CODE    000AH     0001H     UNIT         ?PR?_?OSTIMETICKHOOK?OS_CPU_C
            CODE    000BH     0003H     ABSOLUTE     
            CODE    000EH     035CH     UNIT         ?PR?PRINTF?PRINTF
            CODE    036AH     0318H     UNIT         ?C?LIB_CODE
            CODE    0682H     0263H     UNIT         ?PR?_?OSTCBINIT?OS_CORE
            CODE    08E5H     01B6H     UNIT         ?PR?_?OSTASKSTKINIT?OS_CPU_C
            CODE    0A9BH     01A3H     UNIT         ?PR?_?OSTIMEDLYHMSM?OS_TIME
            CODE    0C3EH     018FH     UNIT         ?PR?_?OSINIT?OS_CORE
            CODE    0DCDH     0137H     UNIT         ?PR?_?OSTASKCREATE?OS_TASK
            CODE    0F04H     012FH     UNIT         ?PR?_?OSTIMETICK?OS_CORE
            CODE    1033H     0110H     UNIT         ?C_INITSEG
            CODE    1143H     00F5H     UNIT         ?PR?_?OSTIMEDLYRESUME?OS_TIME
            CODE    1238H     009DH     UNIT         ?PR?_?OSTASKQUERY?OS_TASK
            CODE    12D5H     0091H     UNIT         ?PR?_?OSTIMEDLY?OS_TIME
            CODE    1366H     0090H     UNIT         ?PR?_?OSINTEXIT?OS_CORE
            CODE    13F6H     008FH     UNIT         ?C_C51STARTUP
            CODE    1485H     008FH     UNIT         ?PR?_?OSSCHED?OS_CORE
            CODE    1514H     0077H     UNIT         ?PR?OSCTXSW?OS_CPU_A
            CODE    158BH     006FH     UNIT         ?PR?_?OSSTART?OS_CORE
            CODE    15FAH     005BH     UNIT         ?PR?OSSTARTHIGHRDY?OS_CPU_A
            CODE    1655H     0047H     UNIT         ?PR?OSTICKISR?OS_CPU_C
            CODE    169CH     003FH     UNIT         ?PR?MAIN?EX1
            CODE    16DBH     003EH     UNIT         ?PR?_?OSTASKIDLE?OS_CORE
            CODE    1719H     0035H     UNIT         ?PR?_?TASK1?EX1
            CODE    174EH     0035H     UNIT         ?PR?_?TASK2?EX1
            CODE    1783H     002BH     UNIT         ?PR?_?OSSCHEDUNLOCK?OS_CORE
            CODE    17AEH     0029H     UNIT         ?PR?_?OSTIMEGET?OS_TIME
            CODE    17D7H     0027H     UNIT         ?PR?PUTCHAR?PUTCHAR
            CODE    17FEH     0020H     UNIT         ?PR?_?OSTIMESET?OS_TIME
            CODE    181EH     001EH     UNIT         ?PR?_?OSTASKCREATEHOOK?OS_CPU_C
            CODE    183CH     001EH     UNIT         ?PR?_?OSTASKDELHOOK?OS_CPU_C
            CODE    185AH     0010H     UNIT         ?PR?_?OSSCHEDLOCK?OS_CORE
            CODE    186AH     0010H     UNIT         ?PR?SERIALINITIAL?EX1
            CODE    187AH     000DH     UNIT         ?CO?EX1
            CODE    1887H     000CH     UNIT         ?PR?INTERRUPTINITIAL?EX1
            CODE    1893H     000BH     UNIT         ?PR?_?OSINTENTER?OS_CORE
            CODE    189EH     000AH     UNIT         ?PR?OSINTCTXSW?OS_CPU_A
            CODE    18A8H     0001H     UNIT         ?PR?_?OSDUMMY?OS_TASK



OVERLAY MAP OF MODULE:   ex1 (OS_CPU_C)


SEGMENT                                    BIT_GROUP          DATA_GROUP 
  +--> CALLED SEGMENT                   START    LENGTH     START    LENGTH
---------------------------------------------------------------------------
?PR?OSTICKISR?OS_CPU_C                  -----    -----      -----    -----
  +--> ?PR?_?OSINTENTER?OS_CORE
  +--> ?PR?_?OSTIMETICK?OS_CORE
BL51 BANKED LINKER/LOCATER V5.01                                                      11/28/2003  21:21:30  PAGE 3


  +--> ?PR?_?OSINTEXIT?OS_CORE

?PR?_?OSTIMETICK?OS_CORE                -----    -----      -----    -----
  +--> ?PR?_?OSTIMETICKHOOK?OS_CPU_C

?PR?_?OSINTEXIT?OS_CORE                 -----    -----      -----    -----
  +--> ?PR?OSINTCTXSW?OS_CPU_A

?PR?OSINTCTXSW?OS_CPU_A                 -----    -----      -----    -----
  +--> ?PR?OSCTXSW?OS_CPU_A

?PR?OSCTXSW?OS_CPU_A                    -----    -----      -----    -----
  +--> ?PR?_?OSTASKSWHOOK?OS_CPU_C
  +--> ?PR?OSSTARTHIGHRDY?OS_CPU_A

*** NEW ROOT ***************************************************

?C_C51STARTUP                           -----    -----      -----    -----
  +--> ?PR?MAIN?EX1
  +--> ?C_INITSEG

?PR?MAIN?EX1                            -----    -----      -----    -----
  +--> ?PR?SERIALINITIAL?EX1
  +--> ?PR?INTERRUPTINITIAL?EX1
  +--> ?PR?_?OSINIT?OS_CORE
  +--> ?CO?EX1
  +--> ?PR?PRINTF?PRINTF
  +--> ?PR?_?TASK1?EX1
  +--> ?PR?_?OSTASKCREATE?OS_TASK
  +--> ?PR?_?TASK2?EX1
  +--> ?PR?_?OSSTART?OS_CORE

?PR?_?OSINIT?OS_CORE                    -----    -----      -----    -----
  +--> ?PR?_?OSTASKIDLE?OS_CORE
  +--> ?PR?_?OSTASKCREATE?OS_TASK

?PR?_?OSTASKCREATE?OS_TASK              -----    -----      -----    -----
  +--> ?PR?_?OSTASKSTKINIT?OS_CPU_C
  +--> ?PR?_?OSTCBINIT?OS_CORE
  +--> ?PR?_?OSTASKCREATEHOOK?OS_CPU_C
  +--> ?PR?_?OSSCHED?OS_CORE

?PR?_?OSSCHED?OS_CORE                   -----    -----      -----    -----
  +--> ?PR?OSCTXSW?OS_CPU_A

?PR?PRINTF?PRINTF                       0020H.0  0001H.1    0008H    0014H
  +--> ?PR?PUTCHAR?PUTCHAR

?PR?_?TASK1?EX1                         -----    -----      -----    -----
  +--> ?PR?_?OSTIMEDLYHMSM?OS_TIME
  +--> ?CO?EX1
  +--> ?PR?PRINTF?PRINTF

?PR?_?OSTIMEDLYHMSM?OS_TIME             -----    -----      -----    -----
  +--> ?PR?_?OSTIMEDLY?OS_TIME

?PR?_?OSTIMEDLY?OS_TIME                 -----    -----      -----    -----
BL51 BANKED LINKER/LOCATER V5.01                                                      11/28/2003  21:21:30  PAGE 4


  +--> ?PR?_?OSSCHED?OS_CORE

?PR?_?TASK2?EX1                         -----    -----      -----    -----
  +--> ?PR?_?OSTIMEDLYHMSM?OS_TIME
  +--> ?CO?EX1
  +--> ?PR?PRINTF?PRINTF

?PR?_?OSSTART?OS_CORE                   -----    -----      -----    -----
  +--> ?PR?OSSTARTHIGHRDY?OS_CPU_A



SYMBOL TABLE OF MODULE:  ex1 (OS_CPU_C)

  VALUE           TYPE          NAME
  ----------------------------------

  -------         MODULE        OS_CPU_C
  C:0000H         SYMBOL        _ICE_DUMMY_
  C:183CH         PUBLIC        _?OSTaskDelHook
  C:0009H         PUBLIC        _?OSTaskStatHook
  C:1655H         PUBLIC        OSTickISR
  C:08E5H         PUBLIC        _?OSTaskStkInit
  C:0008H         PUBLIC        _?OSTaskSwHook
  C:181EH         PUBLIC        _?OSTaskCreateHook
  D:008CH         PUBLIC        TH0
  D:008AH         PUBLIC        TL0
  C:000AH         PUBLIC        _?OSTimeTickHook
  -------         PROC          _?OSTASKSTKINIT
  i:0002H         SYMBOL        task
  i:0004H         SYMBOL        ppdata
  i:0006H         SYMBOL        ptos
  i:0008H         SYMBOL        opt
  -------         DO            
  i:0000H         SYMBOL        stk
  -------         ENDDO         
  C:08E5H         LINE#         69
  C:090AH         LINE#         73
  C:091EH         LINE#         74
  C:0932H         LINE#         76
  C:0943H         LINE#         77
  C:0955H         LINE#         79
  C:0968H         LINE#         80
  C:0981H         LINE#         81
  C:099BH         LINE#         82
  C:09AEH         LINE#         83
  C:09C1H         LINE#         84
  C:09D4H         LINE#         85
  C:09E7H         LINE#         86
  C:09F9H         LINE#         87
  C:0A0BH         LINE#         88
  C:0A1EH         LINE#         89
  C:0A31H         LINE#         90
  C:0A44H         LINE#         91
  C:0A57H         LINE#         92
  C:0A6AH         LINE#         93
  C:0A7DH         LINE#         94
BL51 BANKED LINKER/LOCATER V5.01                                                      11/28/2003  21:21:30  PAGE 5


  C:0A90H         LINE#         96
  C:0A94H         LINE#         97
  -------         ENDPROC       _?OSTASKSTKINIT
  -------         PROC          OSTICKISR
  C:1655H         LINE#         110
  C:1672H         LINE#         112
  C:1675H         LINE#         113
  C:1678H         LINE#         115
  C:167BH         LINE#         116
  C:167EH         LINE#         117
  C:1681H         LINE#         118
  -------         ENDPROC       OSTICKISR
  -------         PROC          _?OSTASKCREATEHOOK
  i:0000H         SYMBOL        ptcb
  C:181EH         LINE#         134
  C:1829H         LINE#         136
  C:1837H         LINE#         137
  -------         ENDPROC       _?OSTASKCREATEHOOK
  -------         PROC          _?OSTASKDELHOOK
  i:0000H         SYMBOL        ptcb
  C:183CH         LINE#         151
  C:1847H         LINE#         153
  C:1855H         LINE#         154
  -------         ENDPROC       _?OSTASKDELHOOK
  -------         PROC          _?OSTASKSWHOOK
  C:0008H         LINE#         171
  C:0008H         LINE#         173
  -------         ENDPROC       _?OSTASKSWHOOK
  -------         PROC          _?OSTASKSTATHOOK
  C:0009H         LINE#         185
  C:0009H         LINE#         187
  -------         ENDPROC       _?OSTASKSTATHOOK
  -------         PROC          _?OSTIMETICKHOOK
  C:000AH         LINE#         200
  C:000AH         LINE#         202
  -------         ENDPROC       _?OSTIMETICKHOOK
  -------         ENDMOD        OS_CPU_C

  -------         MODULE        OS_CPU_A
  C:15FAH         SEGMENT       ?PR?OSSTARTHIGHRDY?OS_CPU_A
  C:1514H         SEGMENT       ?PR?OSCTXSW?OS_CPU_A
  C:189EH         SEGMENT       ?PR?OSINTCTXSW?OS_CPU_A
  I:0022H         SEGMENT       ?STACK
  C:1514H         PUBLIC        OSCTXSW
  C:189EH         PUBLIC        OSINTCTXSW
  C:15FAH         PUBLIC        OSSTARTHIGHRDY
  D:00E0H         SYMBOL        ACC
  D:00F0H         SYMBOL        B
  D:0083H         SYMBOL        DPH
  D:0082H         SYMBOL        DPL
  B:00A8H.7       SYMBOL        EA
  C:1632H         SYMBOL        OSCPUARSTHARDSTK
  C:1605H         SYMBOL        OSCPUARSTSTK
  C:155BH         SYMBOL        OSCPUASAVESTK
  C:162AH         SYMBOL        OSCPUASMLTRSTOVER
  C:1624H         SYMBOL        OSCPUASMLTRSTSTK
  C:154AH         SYMBOL        OSCPUASMLTSAVE
BL51 BANKED LINKER/LOCATER V5.01                                                      11/28/2003  21:21:30  PAGE 6


  C:1551H         SYMBOL        OSCPUASMLTSAVEOVER
  C:152EH         SYMBOL        OSCPUAUNIFORMCTXSW
  N:0000H         SYMBOL        OS_CPU_A
  D:00D0H         SYMBOL        PSW
  D:0081H         SYMBOL        SP
  I:0022H         SYMBOL        STKBOTTOM
  B:0088H.4       SYMBOL        TR0
  C:15FAH         LINE#         110
  C:15FDH         LINE#         111
  C:1600H         LINE#         112
  C:1602H         LINE#         113
  C:1603H         LINE#         118
  C:1605H         LINE#         128
  C:1608H         LINE#         129
  C:160BH         LINE#         130
  C:160CH         LINE#         131
  C:160DH         LINE#         132
  C:160EH         LINE#         133
  C:160FH         LINE#         134
  C:1611H         LINE#         135
  C:1613H         LINE#         138
  C:1614H         LINE#         139
  C:1615H         LINE#         140
  C:1616H         LINE#         141
  C:1617H         LINE#         142
  C:1619H         LINE#         143
  C:161BH         LINE#         150
  C:161CH         LINE#         151
  C:161EH         LINE#         154
  C:1620H         LINE#         155
  C:1621H         LINE#         156
  C:1622H         LINE#         157
  C:1623H         LINE#         158
  C:1624H         LINE#         160
  C:1625H         LINE#         161
  C:1626H         LINE#         162
  C:1627H         LINE#         163
  C:1628H         LINE#         164
  C:162AH         LINE#         168
  C:162BH         LINE#         169
  C:162CH         LINE#         170
  C:162EH         LINE#         171
  C:162FH         LINE#         172
  C:1630H         LINE#         173
  C:1632H         LINE#         179
  C:1633H         LINE#         180
  C:1634H         LINE#         181
  C:1635H         LINE#         182
  C:1636H         LINE#         183
  C:1638H         LINE#         186
  C:163AH         LINE#         187
  C:163CH         LINE#         188
  C:163EH         LINE#         189
  C:1640H         LINE#         190
  C:1642H         LINE#         191
  C:1644H         LINE#         192
  C:1646H         LINE#         193
BL51 BANKED LINKER/LOCATER V5.01                                                      11/28/2003  21:21:30  PAGE 7


  C:1648H         LINE#         194
  C:164AH         LINE#         195
  C:164CH         LINE#         196
  C:164EH         LINE#         197
  C:1650H         LINE#         198
  C:1652H         LINE#         200
  C:1654H         LINE#         201
  C:1514H         LINE#         215
  C:1516H         LINE#         216
  C:1518H         LINE#         217
  C:151AH         LINE#         218
  C:151CH         LINE#         219
  C:151EH         LINE#         220
  C:1520H         LINE#         221
  C:1522H         LINE#         222
  C:1524H         LINE#         223
  C:1526H         LINE#         224
  C:1528H         LINE#         225
  C:152AH         LINE#         226
  C:152CH         LINE#         227
  C:152EH         LINE#         239
  C:1531H         LINE#         240
  C:1534H         LINE#         241
  C:1535H         LINE#         242
  C:1536H         LINE#         243
  C:1537H         LINE#         244
  C:1538H         LINE#         245
  C:153AH         LINE#         246
  C:153CH         LINE#         249
  C:153DH         LINE#         250
  C:153EH         LINE#         251
  C:153FH         LINE#         252
  C:1540H         LINE#         253
  C:1542H         LINE#         254
  C:1544H         LINE#         262
  C:1546H         LINE#         263
  C:1547H         LINE#         266
  C:1549H         LINE#         267
  C:154AH         LINE#         269
  C:154BH         LINE#         270
  C:154CH         LINE#         271
  C:154DH         LINE#         272
  C:154EH         LINE#         273
  C:1551H         LINE#         277
  C:1552H         LINE#         278
  C:1554H         LINE#         279
  C:1555H         LINE#         280
  C:1557H         LINE#         281
  C:1558H         LINE#         285
  C:1559H         LINE#         286
  C:155BH         LINE#         288
  C:155CH         LINE#         289
  C:155DH         LINE#         290
  C:155EH         LINE#         291
  C:155FH         LINE#         292
  C:1561H         LINE#         298
  C:1564H         LINE#         304
BL51 BANKED LINKER/LOCATER V5.01                                                      11/28/2003  21:21:30  PAGE 8


  C:1567H         LINE#         305
  C:156AH         LINE#         306
  C:156BH         LINE#         307
  C:156CH         LINE#         308
  C:156DH         LINE#         309
  C:156EH         LINE#         310
  C:156FH         LINE#         312
  C:1572H         LINE#         313
  C:1575H         LINE#         314
  C:1576H         LINE#         315
  C:1577H         LINE#         316
  C:1578H         LINE#         317
  C:1579H         LINE#         318
  C:157AH         LINE#         324
  C:157DH         LINE#         325
  C:1580H         LINE#         326
  C:1581H         LINE#         328
  C:1584H         LINE#         329
  C:1587H         LINE#         330
  C:1588H         LINE#         335
  C:189EH         LINE#         346
  C:18A0H         LINE#         347
  C:18A1H         LINE#         348
  C:18A3H         LINE#         349
  C:18A5H         LINE#         351
  -------         ENDMOD        OS_CPU_A

  -------         MODULE        ?C_STARTUP
  C:13F6H         SEGMENT       ?C_C51STARTUP
  I:0022H         SEGMENT       ?STACK
  C:0000H         PUBLIC        ?C_STARTUP
  D:00E0H         SYMBOL        ACC
  D:00F0H         SYMBOL        B
  D:0083H         SYMBOL        DPH
  D:0082H         SYMBOL        DPL
  N:0001H         SYMBOL        IBPSTACK
  N:0100H         SYMBOL        IBPSTACKTOP
  N:0080H         SYMBOL        IDATALEN
  C:13F9H         SYMBOL        IDATALOOP
  N:0000H         SYMBOL        PBPSTACK
  N:8000H         SYMBOL        PBPSTACKTOP
  N:0000H         SYMBOL        PDATALEN
  N:0000H         SYMBOL        PDATASTART
  N:0000H         SYMBOL        PPAGE
  N:0000H         SYMBOL        PPAGEENABLE
  D:0081H         SYMBOL        SP
  C:13F6H         SYMBOL        STARTUP1
  N:0000H         SYMBOL        XBPSTACK
  N:8000H         SYMBOL        XBPSTACKTOP
  N:0000H         SYMBOL        XDATALEN
  N:0000H         SYMBOL        XDATASTART
  C:0000H         LINE#         88
  C:13F6H         LINE#         95
  C:13F8H         LINE#         96
  C:13F9H         LINE#         97
  C:13FAH         LINE#         98
  C:13FCH         LINE#         132
BL51 BANKED LINKER/LOCATER V5.01                                                      11/28/2003  21:21:30  PAGE 9


  C:13FFH         LINE#         147
  C:1402H         LINE#         151
  -------         ENDMOD        ?C_STARTUP

  -------         MODULE        OS_CORE
  C:0000H         SYMBOL        _ICE_DUMMY_
  X:0000H         PUBLIC        OSRdyGrp
  B:00A8H.7       PUBLIC        EA
  X:0001H         PUBLIC        OSRunning
  C:1366H         PUBLIC        _?OSIntExit
  X:0002H         PUBLIC        OSLockNesting
  X:0003H         PUBLIC        OSTCBList
  C:1783H         PUBLIC        _?OSSchedUnlock
  X:0005H         SYMBOL        OSTCBTbl
  X:012BH         PUBLIC        OSTCBFreeList
  X:012DH         PUBLIC        OSTCBCur
  X:012FH         PUBLIC        OSUnMapTbl
  C:1485H         PUBLIC        _?OSSched
  C:0003H         PUBLIC        _?OSVersion
  X:022FH         PUBLIC        OSIntNesting
  X:0230H         PUBLIC        OSTCBHighRdy
  C:0682H         PUBLIC        _?OSTCBInit
  X:0232H         PUBLIC        OSTime
  C:185AH         PUBLIC        _?OSSchedLock
  X:0236H         PUBLIC        OSTCBPrioTbl
  X:02B6H         SYMBOL        OSIntExitY
  X:02B7H         PUBLIC        OSCtxSwCtr
  X:02BBH         PUBLIC        OSEventTbl
  X:02D7H         PUBLIC        OSEventFreeList
  X:02D9H         PUBLIC        OSIdleCtr
  C:158BH         PUBLIC        _?OSStart
  C:16DBH         PUBLIC        _?OSTaskIdle
  C:0C3EH         PUBLIC        _?OSInit
  C:0F04H         PUBLIC        _?OSTimeTick
  X:02DDH         PUBLIC        OSTaskCtr
  X:02DEH         PUBLIC        OSMapTbl
  X:02E6H         PUBLIC        OSPrioCur
  X:02E7H         SYMBOL        OSTaskIdleStk
  C:1893H         PUBLIC        _?OSIntEnter
  X:03DFH         PUBLIC        OSPrioHighRdy
  X:03E0H         PUBLIC        OSRdyTbl
  -------         PROC          _?OSINIT
  -------         DO            
  i:0000H         SYMBOL        i
  -------         ENDDO         
  C:0C3EH         LINE#         225
  C:0C42H         LINE#         230
  C:0C4CH         LINE#         231
  C:0C51H         LINE#         232
  C:0C55H         LINE#         236
  C:0C59H         LINE#         238
  C:0C5DH         LINE#         239
  C:0C67H         LINE#         245
  C:0C71H         LINE#         248
  C:0C76H         LINE#         249
  C:0C88H         LINE#         250
  C:0C97H         LINE#         251
BL51 BANKED LINKER/LOCATER V5.01                                                      11/28/2003  21:21:30  PAGE 10


  C:0CA2H         LINE#         254
  C:0CA7H         LINE#         255
  C:0CABH         LINE#         256
  C:0CB1H         LINE#         257
  C:0CB7H         LINE#         258
  C:0CBDH         LINE#         261
  C:0CD1H         LINE#         262
  C:0CE6H         LINE#         263
  C:0CF1H         LINE#         266
  C:0D04H         LINE#         267
  C:0D36H         LINE#         268
  C:0D41H         LINE#         269
  C:0D48H         LINE#         270
  C:0D52H         LINE#         274
  C:0D65H         LINE#         275
  C:0D97H         LINE#         276
  C:0DA2H         LINE#         277
  C:0DA9H         LINE#         278
  C:0DB3H         LINE#         318
  C:0DC8H         LINE#         359
  -------         ENDPROC       _?OSINIT
  -------         PROC          _?OSINTENTER
  C:1893H         LINE#         384
  C:1893H         LINE#         386
  C:1895H         LINE#         387
  C:189BH         LINE#         388
  C:189DH         LINE#         389
  -------         ENDPROC       _?OSINTENTER
  -------         PROC          _?OSINTEXIT
  C:1366H         LINE#         410
  C:1366H         LINE#         412
  C:1368H         LINE#         413
  C:1378H         LINE#         414
  C:138AH         LINE#         415
  C:13AFH         LINE#         416
  C:13B6H         LINE#         417
  C:13D1H         LINE#         418
  C:13F0H         LINE#         419
  C:13F3H         LINE#         420
  C:13F3H         LINE#         421
  C:13F3H         LINE#         422
  C:13F5H         LINE#         423
  -------         ENDPROC       _?OSINTEXIT
  -------         PROC          _?OSSCHED
  -------         DO            
  i:0000H         SYMBOL        y
  -------         ENDDO         
  C:1485H         LINE#         442
  C:1487H         LINE#         447
  C:1489H         LINE#         448
  C:1495H         LINE#         449
  C:14A6H         LINE#         450
  C:14CBH         LINE#         451
  C:14D2H         LINE#         452
  C:14EDH         LINE#         453
  C:150CH         LINE#         454
  C:150FH         LINE#         455
BL51 BANKED LINKER/LOCATER V5.01                                                      11/28/2003  21:21:30  PAGE 11


  C:150FH         LINE#         456
  C:150FH         LINE#         457
  C:1511H         LINE#         458
  -------         ENDPROC       _?OSSCHED
  -------         PROC          _?OSSCHEDLOCK
  C:185AH         LINE#         476
  C:185AH         LINE#         478
  C:1861H         LINE#         479
  C:1863H         LINE#         480
  C:1867H         LINE#         481
  C:1869H         LINE#         482
  C:1869H         LINE#         483
  -------         ENDPROC       _?OSSCHEDLOCK
  -------         PROC          _?OSSCHEDUNLOCK
  C:1783H         LINE#         500
  C:1783H         LINE#         502
  C:178BH         LINE#         503
  C:178DH         LINE#         504
  C:1794H         LINE#         505
  C:1797H         LINE#         506
  C:17A3H         LINE#         507
  C:17A5H         LINE#         508
  C:17A8H         LINE#         509
  C:17A8H         LINE#         510
  C:17AAH         LINE#         511
  C:17AAH         LINE#         512
  C:17ABH         LINE#         513
  C:17ADH         LINE#         514
  C:17ADH         LINE#         515
  C:17ADH         LINE#         516
  -------         ENDPROC       _?OSSCHEDUNLOCK
  -------         PROC          _?OSSTART
  -------         DO            
  i:0000H         SYMBOL        y
  i:0001H         SYMBOL        x
  -------         ENDDO         
  C:158BH         LINE#         537
  C:158FH         LINE#         543
  C:1595H         LINE#         544
  C:15A6H         LINE#         545
  C:15C0H         LINE#         546
  C:15CEH         LINE#         547
  C:15D2H         LINE#         548
  C:15EAH         LINE#         549
  C:15F2H         LINE#         550
  C:15F5H         LINE#         551
  C:15F5H         LINE#         552
  -------         ENDPROC       _?OSSTART
  -------         PROC          _?OSTASKIDLE
  i:0000H         SYMBOL        ppdata
  C:16DBH         LINE#         602
  C:16E6H         LINE#         604
  C:16F4H         LINE#         605
  C:16F4H         LINE#         606
  C:16F6H         LINE#         607
  C:1715H         LINE#         608
  C:1717H         LINE#         609
BL51 BANKED LINKER/LOCATER V5.01                                                      11/28/2003  21:21:30  PAGE 12


  -------         ENDPROC       _?OSTASKIDLE
  -------         PROC          _?OSTCBINIT
  i:0002H         SYMBOL        prio
  i:0003H         SYMBOL        ptos
  i:0005H         SYMBOL        pbos
  i:0007H         SYMBOL        id
  i:0009H         SYMBOL        stk_size
  i:000BH         SYMBOL        pext
  i:000DH         SYMBOL        opt
  -------         DO            
  i:0000H         SYMBOL        ptcb
  -------         ENDDO         
  C:0682H         LINE#         716
  C:06A2H         LINE#         721
  C:06A4H         LINE#         724
  C:06B3H         LINE#         725
  C:06BEH         LINE#         726
  C:06D7H         LINE#         727
  C:06D9H         LINE#         730
  C:06EBH         LINE#         731
  C:0705H         LINE#         732
  C:0716H         LINE#         733
  C:0729H         LINE#         742
  C:073DH         LINE#         743
  C:0751H         LINE#         744
  C:0765H         LINE#         745
  C:0779H         LINE#         746
  C:078DH         LINE#         754
  C:07A5H         LINE#         755
  C:07D1H         LINE#         756
  C:07EBH         LINE#         757
  C:0817H         LINE#         767
  C:0819H         LINE#         770
  C:082AH         LINE#         773
  C:0844H         LINE#         774
  C:0857H         LINE#         775
  C:085BH         LINE#         776
  C:086FH         LINE#         777
  C:086FH         LINE#         778
  C:087EH         LINE#         781
  C:089AH         LINE#         782
  C:08D4H         LINE#         783
  C:08D6H         LINE#         784
  C:08DAH         LINE#         785
  C:08DAH         LINE#         788
  C:08DCH         LINE#         789
  C:08DEH         LINE#         790
  C:08DEH         LINE#         791
  -------         ENDPROC       _?OSTCBINIT
  -------         PROC          _?OSTIMETICK
  -------         DO            
  i:0000H         SYMBOL        ptcb
  -------         ENDDO         
  C:0F04H         LINE#         807
  C:0F08H         LINE#         812
  C:0F0BH         LINE#         813
  C:0F1AH         LINE#         814
BL51 BANKED LINKER/LOCATER V5.01                                                      11/28/2003  21:21:30  PAGE 13


  C:0F34H         LINE#         815
  C:0F36H         LINE#         816
  C:0F4FH         LINE#         817
  C:0F6FH         LINE#         818
  C:0F82H         LINE#         819
  C:0FA1H         LINE#         820
  C:0FD8H         LINE#         821
  C:0FDAH         LINE#         822
  C:0FF0H         LINE#         823
  C:0FF0H         LINE#         824
  C:0FF0H         LINE#         825
  C:0FF0H         LINE#         826
  C:1006H         LINE#         827
  C:1008H         LINE#         828
  C:100BH         LINE#         829
  C:100DH         LINE#         830
  C:102CH         LINE#         831
  C:102EH         LINE#         832
  -------         ENDPROC       _?OSTIMETICK
  -------         PROC          _?OSVERSION
  C:0003H         LINE#         848
  C:0003H         LINE#         850
  C:0007H         LINE#         851
  -------         ENDPROC       _?OSVERSION
  -------         ENDMOD        OS_CORE

  -------         MODULE        OS_MBOX
  C:0000H         SYMBOL        _ICE_DUMMY_
  -------         ENDMOD        OS_MBOX

  -------         MODULE        OS_MEM
  C:0000H         SYMBOL        _ICE_DUMMY_
  -------         ENDMOD        OS_MEM

  -------         MODULE        OS_Q
  C:0000H         SYMBOL        _ICE_DUMMY_
  -------         ENDMOD        OS_Q

  -------         MODULE        OS_SEM
  C:0000H         SYMBOL        _ICE_DUMMY_
  -------         ENDMOD        OS_SEM

  -------         MODULE        OS_TASK
  C:0000H         SYMBOL        _ICE_DUMMY_
  B:00A8H.7       PUBLIC        EA
  C:0DCDH         PUBLIC        _?OSTaskCreate
  C:18A8H         SYMBOL        _?OSDummy
  C:1238H         PUBLIC        _?OSTaskQuery
  -------         PROC          _?OSDUMMY
  C:18A8H         LINE#         43
  C:18A8H         LINE#         45
  -------         ENDPROC       _?OSDUMMY
  -------         PROC          _?OSTASKCREATE
  i:0003H         SYMBOL        task
  i:0005H         SYMBOL        ppdata
  i:0007H         SYMBOL        ptos
  i:0009H         SYMBOL        prio
BL51 BANKED LINKER/LOCATER V5.01                                                      11/28/2003  21:21:30  PAGE 14


  -------         DO            
  i:0000H         SYMBOL        psp
  i:0002H         SYMBOL        err
  -------         ENDDO         
  C:0DCDH         LINE#         173
  C:0DF4H         LINE#         178
  C:0E00H         LINE#         179
  C:0E05H         LINE#         180
  C:0E05H         LINE#         181
  C:0E07H         LINE#         182
  C:0E1DH         LINE#         183
  C:0E33H         LINE#         185
  C:0E35H         LINE#         186
  C:0E67H         LINE#         187
  C:0EA8H         LINE#         188
  C:0EAAH         LINE#         189
  C:0EACH         LINE#         190
  C:0EB2H         LINE#         191
  C:0ECBH         LINE#         192
  C:0ECDH         LINE#         193
  C:0ED3H         LINE#         194
  C:0ED6H         LINE#         195
  C:0ED6H         LINE#         196
  C:0ED8H         LINE#         197
  C:0EDAH         LINE#         198
  C:0EEFH         LINE#         199
  C:0EF1H         LINE#         200
  C:0EF1H         LINE#         201
  C:0EF9H         LINE#         202
  C:0EF9H         LINE#         203
  C:0EFBH         LINE#         204
  C:0EFDH         LINE#         205
  C:0EFDH         LINE#         206
  -------         ENDPROC       _?OSTASKCREATE
  -------         PROC          _?OSTASKQUERY
  i:0002H         SYMBOL        prio
  i:0003H         SYMBOL        ppdata
  -------         DO            
  i:0000H         SYMBOL        ptcb
  -------         ENDDO         
  C:1238H         LINE#         699
  C:124DH         LINE#         704
  C:125CH         LINE#         705
  C:1260H         LINE#         706
  C:1260H         LINE#         707
  C:1262H         LINE#         708
  C:126AH         LINE#         709
  C:127FH         LINE#         710
  C:127FH         LINE#         711
  C:129EH         LINE#         712
  C:12A0H         LINE#         713
  C:12A4H         LINE#         714
  C:12A4H         LINE#         715
  C:12CAH         LINE#         716
  C:12CCH         LINE#         717
  C:12CEH         LINE#         718
  -------         ENDPROC       _?OSTASKQUERY
BL51 BANKED LINKER/LOCATER V5.01                                                      11/28/2003  21:21:30  PAGE 15


  -------         ENDMOD        OS_TASK

  -------         MODULE        OS_TIME
  C:0000H         SYMBOL        _ICE_DUMMY_
  C:12D5H         PUBLIC        _?OSTimeDly
  C:17FEH         PUBLIC        _?OSTimeSet
  B:00A8H.7       PUBLIC        EA
  C:0A9BH         PUBLIC        _?OSTimeDlyHMSM
  C:1143H         PUBLIC        _?OSTimeDlyResume
  C:17AEH         PUBLIC        _?OSTimeGet
  -------         PROC          _?OSTIMEDLY
  i:0000H         SYMBOL        ticks
  C:12D5H         LINE#         37
  C:12E0H         LINE#         39
  C:12EDH         LINE#         40
  C:12EFH         LINE#         41
  C:1324H         LINE#         42
  C:1341H         LINE#         43
  C:1341H         LINE#         44
  C:135CH         LINE#         45
  C:135EH         LINE#         46
  C:1361H         LINE#         47
  C:1361H         LINE#         48
  -------         ENDPROC       _?OSTIMEDLY
  -------         PROC          _?OSTIMEDLYHMSM
  i:0006H         SYMBOL        hours
  i:0007H         SYMBOL        minutes
  i:0008H         SYMBOL        seconds
  i:0009H         SYMBOL        milli
  -------         DO            
  i:0000H         SYMBOL        ticks
  i:0004H         SYMBOL        loops
  -------         ENDDO         
  C:0A9BH         LINE#         75
  C:0AB3H         LINE#         81
  C:0AE5H         LINE#         82
  C:0AF1H         LINE#         83
  C:0AF6H         LINE#         84
  C:0AF6H         LINE#         85
  C:0B01H         LINE#         86
  C:0B06H         LINE#         87
  C:0B06H         LINE#         88
  C:0B16H         LINE#         89
  C:0B1BH         LINE#         90
  C:0B1BH         LINE#         94
  C:0BCEH         LINE#         95
  C:0BEAH         LINE#         96
  C:0BF9H         LINE#         97
  C:0C05H         LINE#         98
  C:0C15H         LINE#         99
  C:0C1CH         LINE#         100
  C:0C23H         LINE#         101
  C:0C2FH         LINE#         102
  C:0C31H         LINE#         103
  C:0C35H         LINE#         104
  C:0C35H         LINE#         105
  C:0C37H         LINE#         106
BL51 BANKED LINKER/LOCATER V5.01                                                      11/28/2003  21:21:30  PAGE 16


  C:0C37H         LINE#         107
  -------         ENDPROC       _?OSTIMEDLYHMSM
  -------         PROC          _?OSTIMEDLYRESUME
  i:0002H         SYMBOL        prio
  -------         DO            
  i:0000H         SYMBOL        ptcb
  -------         ENDDO         
  C:1143H         LINE#         133
  C:114DH         LINE#         138
  C:1158H         LINE#         139
  C:115DH         LINE#         140
  C:115DH         LINE#         141
  C:115FH         LINE#         142
  C:1175H         LINE#         143
  C:1182H         LINE#         144
  C:119BH         LINE#         145
  C:11B1H         LINE#         146
  C:11C4H         LINE#         147
  C:11E3H         LINE#         148
  C:121AH         LINE#         149
  C:121CH         LINE#         150
  C:121FH         LINE#         151
  C:1221H         LINE#         152
  C:1223H         LINE#         153
  C:1223H         LINE#         154
  C:1227H         LINE#         155
  C:1227H         LINE#         156
  C:1229H         LINE#         157
  C:122DH         LINE#         158
  C:122DH         LINE#         159
  C:122DH         LINE#         160
  C:122FH         LINE#         161
  C:1231H         LINE#         162
  C:1231H         LINE#         163
  -------         ENDPROC       _?OSTIMEDLYRESUME
  -------         PROC          _?OSTIMEGET
  -------         DO            
  i:0000H         SYMBOL        ticks
  -------         ENDDO         
  C:17AEH         LINE#         178
  C:17B4H         LINE#         183
  C:17B6H         LINE#         184
  C:17C9H         LINE#         185
  C:17CBH         LINE#         186
  C:17D0H         LINE#         187
  -------         ENDPROC       _?OSTIMEGET
  -------         PROC          _?OSTIMESET
  i:0000H         SYMBOL        ticks
  C:17FEH         LINE#         201
  C:1808H         LINE#         203
  C:180AH         LINE#         204
  C:1815H         LINE#         205
  C:1817H         LINE#         206
  -------         ENDPROC       _?OSTIMESET
  -------         ENDMOD        OS_TIME

  -------         MODULE        EX1
BL51 BANKED LINKER/LOCATER V5.01                                                      11/28/2003  21:21:30  PAGE 17


  C:0000H         SYMBOL        _ICE_DUMMY_
  C:1887H         PUBLIC        InterruptInitial
  C:169CH         PUBLIC        main
  D:0087H         PUBLIC        PCON
  C:186AH         PUBLIC        SerialInitial
  D:0098H         PUBLIC        SCON
  D:0089H         PUBLIC        TMOD
  D:0088H         PUBLIC        TCON
  X:03E8H         PUBLIC        Task1Stack
  X:04E0H         PUBLIC        Task2Stack
  B:00A8H.1       PUBLIC        ET0
  D:008CH         PUBLIC        TH0
  D:008DH         PUBLIC        TH1
  D:008AH         PUBLIC        TL0
  C:1719H         PUBLIC        _?Task1
  C:174EH         PUBLIC        _?Task2
  -------         PROC          _?TASK1
  i:0000H         SYMBOL        ppdata
  C:1719H         LINE#         6
  C:1724H         LINE#         8
  C:1732H         LINE#         9
  C:1732H         LINE#         10
  C:1732H         LINE#         11
  C:1743H         LINE#         12
  C:174CH         LINE#         13
  -------         ENDPROC       _?TASK1
  -------         PROC          _?TASK2
  i:0000H         SYMBOL        ppdata
  C:174EH         LINE#         16
  C:1759H         LINE#         18
  C:1767H         LINE#         19
  C:1767H         LINE#         20
  C:1767H         LINE#         21
  C:1778H         LINE#         22
  C:1781H         LINE#         23
  -------         ENDPROC       _?TASK2
  -------         PROC          SERIALINITIAL
  C:186AH         LINE#         25
  C:186AH         LINE#         26
  C:186AH         LINE#         28
  C:186DH         LINE#         29
  C:1870H         LINE#         30
  C:1873H         LINE#         31
  C:1876H         LINE#         32
  C:1879H         LINE#         33
  -------         ENDPROC       SERIALINITIAL
  -------         PROC          INTERRUPTINITIAL
  C:1887H         LINE#         34
  C:1887H         LINE#         35
  C:1887H         LINE#         37
  C:188AH         LINE#         38
  C:188DH         LINE#         39
  C:1890H         LINE#         41
  C:1892H         LINE#         42
  -------         ENDPROC       INTERRUPTINITIAL
  -------         PROC          MAIN
  C:169CH         LINE#         43
BL51 BANKED LINKER/LOCATER V5.01                                                      11/28/2003  21:21:30  PAGE 18


  C:169CH         LINE#         44
  C:169CH         LINE#         45
  C:169FH         LINE#         46
  C:16A2H         LINE#         47
  C:16A5H         LINE#         48
  C:16AEH         LINE#         49
  C:16C3H         LINE#         50
  C:16D8H         LINE#         51
  -------         ENDPROC       MAIN
  -------         ENDMOD        EX1

  -------         MODULE        ?C?COPY
  C:043AH         PUBLIC        ?C?COPY
  -------         ENDMOD        ?C?COPY

  -------         MODULE        ?C?IILDX
  C:0460H         PUBLIC        ?C?IILDX
  -------         ENDMOD        ?C?IILDX

  -------         MODULE        ?C?LMUL
  C:0476H         PUBLIC        ?C?LMUL
  -------         ENDMOD        ?C?LMUL

  -------         MODULE        ?C?ULDIV
  C:0501H         PUBLIC        ?C?ULDIV
  -------         ENDMOD        ?C?ULDIV

  -------         MODULE        ?C?LLDIDATA
  C:0593H         PUBLIC        ?C?LLDIDATA
  -------         ENDMOD        ?C?LLDIDATA

  -------         MODULE        ?C?LSTIDATA
  C:059FH         PUBLIC        ?C?LSTIDATA
  -------         ENDMOD        ?C?LSTIDATA

  -------         MODULE        ?C?LSTXDATA
  C:05ABH         PUBLIC        ?C?LSTXDATA
  -------         ENDMOD        ?C?LSTXDATA

  -------         MODULE        ?C?LSTKXDATA
  C:05B7H         PUBLIC        ?C?LSTKXDATA
  -------         ENDMOD        ?C?LSTKXDATA

  -------         MODULE        ?C?OFFXADD
  C:05E8H         PUBLIC        ?C?OFFXADD
  -------         ENDMOD        ?C?OFFXADD

  -------         MODULE        ?C_IBP
  D:001CH         PUBLIC        ?C_IBP
  -------         ENDMOD        ?C_IBP

  -------         MODULE        PRINTF
  D:0008H         PUBLIC        ?_PRINTF517?BYTE
  D:0008H         PUBLIC        ?_PRINTF?BYTE
  D:0008H         PUBLIC        ?_SPRINTF517?BYTE
  D:0008H         PUBLIC        ?_SPRINTF?BYTE
  C:0070H         PUBLIC        _PRINTF
BL51 BANKED LINKER/LOCATER V5.01                                                      11/28/2003  21:21:30  PAGE 19


  C:0070H         PUBLIC        _PRINTF517
  C:006AH         PUBLIC        _SPRINTF
  C:006AH         PUBLIC        _SPRINTF517
  -------         ENDMOD        PRINTF

  -------         MODULE        ?C?CLDPTR
  C:05F4H         PUBLIC        ?C?CLDPTR
  -------         ENDMOD        ?C?CLDPTR

  -------         MODULE        ?C?CLDOPTR
  C:060DH         PUBLIC        ?C?CLDOPTR
  -------         ENDMOD        ?C?CLDOPTR

  -------         MODULE        ?C?CSTPTR
  C:063AH         PUBLIC        ?C?CSTPTR
  -------         ENDMOD        ?C?CSTPTR

  -------         MODULE        ?C?PLDIIDATA
  C:064CH         PUBLIC        ?C?PLDIIDATA
  -------         ENDMOD        ?C?PLDIIDATA

  -------         MODULE        ?C?CCASE
  C:065CH         PUBLIC        ?C?CCASE
  -------         ENDMOD        ?C?CCASE

  -------         MODULE        PUTCHAR
  C:17D7H         PUBLIC        _PUTCHAR
  -------         ENDMOD        PUTCHAR

*** WARNING L16: UNCALLED SEGMENT, IGNORED FOR OVERLAY PROCESS
    SEGMENT: ?PR?_?OSTASKDELHOOK?OS_CPU_C

*** WARNING L16: UNCALLED SEGMENT, IGNORED FOR OVERLAY PROCESS
    SEGMENT: ?PR?_?OSTASKSTATHOOK?OS_CPU_C

*** WARNING L16: UNCALLED SEGMENT, IGNORED FOR OVERLAY PROCESS
    SEGMENT: ?PR?_?OSSCHEDLOCK?OS_CORE

*** WARNING L16: UNCALLED SEGMENT, IGNORED FOR OVERLAY PROCESS
    SEGMENT: ?PR?_?OSSCHEDUNLOCK?OS_CORE

*** WARNING L16: UNCALLED SEGMENT, IGNORED FOR OVERLAY PROCESS
    SEGMENT: ?PR?_?OSVERSION?OS_CORE

*** WARNING L16: UNCALLED SEGMENT, IGNORED FOR OVERLAY PROCESS
    SEGMENT: ?PR?_?OSDUMMY?OS_TASK

*** WARNING L16: UNCALLED SEGMENT, IGNORED FOR OVERLAY PROCESS
    SEGMENT: ?PR?_?OSTASKQUERY?OS_TASK

*** WARNING L16: UNCALLED SEGMENT, IGNORED FOR OVERLAY PROCESS
    SEGMENT: ?PR?_?OSTIMEDLYRESUME?OS_TIME

*** WARNING L16: UNCALLED SEGMENT, IGNORED FOR OVERLAY PROCESS
    SEGMENT: ?PR?_?OSTIMEGET?OS_TIME

*** WARNING L16: UNCALLED SEGMENT, IGNORED FOR OVERLAY PROCESS
BL51 BANKED LINKER/LOCATER V5.01                                                      11/28/2003  21:21:30  PAGE 20


    SEGMENT: ?PR?_?OSTIMESET?OS_TIME

Program Size: data=31.1 xdata=1496 code=6313
LINK/LOCATE RUN COMPLETE.  10 WARNING(S),  0 ERROR(S)
